:100000000C9444050C94AF050C9492080C94AF0525
:100010000C94AF050C94AF050C94AF050C94AF0590
:100020000C94AF050C94AF050C9408160C94AF0516
:100030000C94D2230C94AF050C94AF050C94AF052F
:100040000C94AF050C94AF050C94AF050C94AF0560
:100050000C94AF050C9427240C94AF050C94AF05B9
:100060000C94AF050C94AF050C94AF050C94AF0540
:100070000C94AF050C94AF050C94AF050C94AF0530
:100080000C94AF050C94AF050C94AF050C94AF0520
:100090000C94AF050C94AF05620A640A700A700AEA
:1000A000700A700A700A700A660A680A6A0A700A98
:1000B000700A640A720A700A700A2C0A620A700ACC
:1000C000700A680A700A700A700A700A700A700A68
:1000D0006A0A620A4E0A700A520A700A700A700AA4
:1000E0002E0A660A700A700A5C0A700A700A700AA0
:1000F000300A6E0A700A500A700A640A700A700A9E
:10010000600A540A700A560A680A700A700A700A6D
:100110005E0A580A700A700A700A700A700A700A39
:10012000700A5A0A700A320A700A700A660A700A5D
:10013000700A6E0A700A700A700A700A700A700AF1
:10014000700A700A700A340A700A700A700A5C0A2F
:10015000700A700A700A700A700A700A700A700ACF
:10016000700A700A360A700A380A3A0A700A700A67
:10017000700A3C0A3E0A400A700A420A440A700A9F
:10018000700A700A6C0A460A700A4A0A480A4C0A3F
:10019000700A700A700A700A6E0A960AA40AB00AF7
:1001A000B00A880AB00AB00AB00AB00AB00AB00AA7
:1001B000B00AB00AB00AB00AB00AB00AB00A8A0A95
:1001C000B00A8C0AB00AB00AB00AB00AA80AB00A8B
:1001D000BF0AA60AB00AB00AB00AB00AB00AB00A4A
:1001E000B00AB00AB00AB00AB00AB00AB00A800A6F
:1001F0009C0A8E0AA00AB00A900AB00A940AB00AB1
:100200009E0A920AA20A980A9A0AB00AB00AB00A8A
:10021000B00AB00AB00AB00A820A840A860AAA0A98
:10022000AC0AB00AB00AB00AAE0A8E0BAC0BB80B1F
:10023000DC0BEC0BF80B140C2B0C4E0C6B0CF60CB3
:10024000220D9B0DCD0DB70DDE0DF00DF80DFE0D41
:10025000020E080E640E660E680E6A0EAA0E720E6C
:10026000720E720E6C0E6E0E700E53147A1472159E
:100270007A147215C614E914721540154F15D21967
:10028000D2190A1A0A1A851A991C991C991CB91AAA
:10029000991C611A611A531C991C681C861C007BEE
:1002A00046010203763A687F6577482B353B6978CB
:1002B000796439141E3C6A7A1D16041A1F3D6B06B8
:1002C0001B070821203E6C2C19091715223F6D11C0
:1002D000050B0A1C23406E7E100D182425416F3635
:1002E0000E0C122726427037380F33132D437175C9
:1002F00034322F2E44727C7D283031744573515036
:100300004A524D492A5466594F5C5F4C4B4E6263CA
:100310005A5D5E60295367585B565761475548429E
:10032000403E3C3A3B456843413F3D2B357E697A30
:10033000790078141E7C6A7B1D16041A1F7F6B06D9
:100340001B070821204D6C2C19091715224A6D1125
:10035000050B0A1C234C6E49100D182425516F36CD
:100360000E0C1227264F7037380F33132D5271752C
:1003700034502F2E4E72397D283065314B735464C2
:10038000586776012A773259745C5F6602036263AC
:100390005A5D5E60295344575B5655614746802934
:1003A0001E1F20212223242526272D2E2A2B141A16
:1003B0000815171C180C12132F302878041607097B
:1003C0000A0B0D0E0F33343579311D1B061905113B
:1003D000103637387D557A2C393A3B3C3D3E3F400C
:1003E00041424353475F6061565C5D5E57595A5BBB
:1003F00062634648324445677B7F65030102525081
:10040000514F68696A6B6C6D6E6F707172580049FC
:100410004C754A4D734B4E767C777E7466547225CC
:100420003032582000623A2530345820006525309B
:10043000325820002146554C4C21200021464621AF
:10044000200077253032582000214353335F463057
:10045000210A00214353335F5245414459210A0088
:10046000214353325F45305F4630210A0021435318
:10047000325F4630210A00214353325F4530210A62
:1004800000214353325F494E4954210A002143530E
:10049000315F45305F25303258210A000A5B4F56E4
:1004A000525D20004C2575200053257520000A4917
:1004B000443A253034582825642920004D6F75733F
:1004C000653A206E6F7420737570706F7274656416
:1004D0000A005225752000572575200057257520E4
:1004E00000572575200058257520004125752000EE
:1004F00049257520005B4348475D20000A5052544F
:100500003A25303258204953523A25303458200089
:100510005B5253545D20000A4552523A25303258FE
:10052000204953523A2530345820000A4B657962ED
:100530006F6172642073746172742E0A000A5553DD
:100540004220636F6E666967757265642E0A000AE1
:100550000A544D4B3A36623731643838312F4C5596
:1005600046410A0A003403490042004D0020005071
:1005700000430020006B006500790062006F00619D
:100580000072006400200063006F006E007600655A
:1005900000720074006500720000000E0374002EEB
:1005A000006D002E006B002E0000000403090409FA
:1005B000027400040100A0320904000001030101DB
:1005C00000092111010001224000070581030800F4
:1005D0000A090401000103000000092111010001C2
:1005E0002236000705820308000A090402000203FC
:1005F00000000009211101000122220007058303E8
:100600002000010705030320000109040300010382
:1006100000000009211101000122390007058403AF
:100620002000011201100100000008EDFEEE1B0188
:10063000000102000105010906A101050719E029D1
:10064000E7150025019508750181020508190129A2
:10065000059505750191029501750391010507192D
:100660000029F71500250195F875018102C00631B2
:10067000FF0974A1010975150026FF009520750872
:1006800081020976150026FF00952075089102C0A9
:1006900005010980A10185021601002637001A8193
:1006A000002AB700751095018100C0050C0901A151
:1006B000018503160100269C021A01002A9C02757E
:1006C0001095018100C005010906A101050719E087
:1006D00029E7150025019508750181029501750826
:1006E00081010508190129059505750191029501FA
:1006F000750391010507190029FF150026FF0095D4
:100700000675088100C0636F6E73756D65723A205F
:10071000253034580A0073797374656D3A2025309A
:1007200034580A000A002530325820006B6579627F
:100730006F6172643A20004C45443A2025303258AB
:100740000A0025583A2530386225730A000A20200D
:1007500030313233343536370A0064656C5F6B658F
:10076000795F6269743A2063616E27742064656CF6
:100770003A20253032580A006164645F6B65795F06
:100780006269743A2063616E2774206164643A2060
:10079000253032580A003F00433E20004C25640AB1
:1007A000000A092D20436F6E736F6C65202D0A457A
:1007B00053432F713A09717569740A000A092D2093
:1007C0004D61676963202D0A643A09646562756743
:1007D0000A783A096465627567206D617472697898
:1007E0000A6B3A096465627567206B6579626F61AF
:1007F00072640A6D3A096465627567206D6F75737E
:10080000650A763A0976657273696F6E0A733A09FA
:100810007374617475730A633A09636F6E736F6CF6
:1008200065206D6F64650A302D343A096C61796515
:1008300072302D34284631302D4634290A506175E6
:10084000733A09626F6F746C6F616465720A6E3A15
:10085000094E4B524F0A003F004E4B524F3A206F09
:1008600066660A004E4B524F3A206F6E0A0074695A
:100870006D65725F72656164333228293A202530D4
:10088000346C580A006B6579626F6172645F6E6BDD
:10089000726F3A2025580A006B6579626F61726445
:1008A0005F69646C653A2025580A006B6579626F50
:1008B0006172645F70726F746F636F6C3A20255859
:1008C0000A00686F73745F6B6579626F6172645F51
:1008D0006C65647328293A2025580A000A092D20DE
:1008E000537461747573202D0A004743433A2035D1
:1008F0002E342E30204156522D4C4942433A20325C
:100900002E302E30204156525F415243483A2061EA
:10091000767235310A004F5054494F4E533A204CAD
:100920005546412045585452414B455920434F4E5E
:10093000534F4C4520434F4D4D414E44204E4B525A
:100940004F204B45594D41505F53454354494F4EFD
:1009500020424F4F544C4F414445525F53495A45F2
:100960000A004255494C443A2036623731643838DF
:1009700031202830343A32373A3330204E6F7620E7
:1009800032322032303230290A005649443A20307F
:10099000784645454428742E6D2E6B2E29205049EB
:1009A000443A203078316265652849424D205043F1
:1009B000206B6579626F61726420636F6E76657219
:1009C00074657229205645523A20307830303031E3
:1009D0000A00444553433A20636F6E766572742073
:1009E00049424D205043206B6579626F61726420EB
:1009F000746F205553420A000A092D205665727300
:100A0000696F6E202D0A000A6D6F7573653A206F4D
:100A100066660A000A6D6F7573653A206F6E0A008C
:100A20000A6B6579626F6172643A206F66660A00CC
:100A30000A6B6579626F6172643A206F6E0A000A10
:100A40006D61747269783A206F66660A000A6D619A
:100A5000747269783A206F6E0A000A64656275677D
:100A60003A206F6E0A000A64656275673A206F6605
:100A7000660A000A0A626F6F746C6F616465722E99
:100A80002E2E2000433E200011241FBECFEFD0E2C7
:100A9000DEBFCDBF04B603FE49C0809188039091AC
:100AA0008903A0918A03B0918B038730904BA740B4
:100AB000B04B09F03BC0109288031092890310924A
:100AC0008A0310928B0314BE0FB6F894A8958091F8
:100AD0006000886180936000109260000FBE1092E9
:100AE000010810920008E3E0F0E089E080935700ED
:100AF000E491E695E370E150E33040F4F0E0EE0F6E
:100B0000FF1FE35DFE4F2081318102C020E030E213
:100B100080E090E0A2E0B0E0821B930BA109B10954
:100B2000B595A79597958795FC01099511E0A0E0EB
:100B3000B1E0EEE5FCE400E00BBF02C007900D92CF
:100B4000A433B107D9F723E0A4E3B1E001C01D92BB
:100B5000A838B207E1F70E946E110C942D260C9470
:100B60000000FF93EF93E0913401F091350130974D
:100B700009F00995EF91FF910895FC01859180306E
:100B800011F0EFDFFBCF0895FF27E0E230E247FFEF
:100B90000CC0419597FF09C0EDE260957095809576
:100BA0009095611D711D811D911D27FF02C021952A
:100BB00030E350E2AA27660F771F881F991FAA1FEC
:100BC000A41710F0A41B63955A95A9F7AA3008F052
:100BD000A95FA05DAF93F39561157105810591053E
:100BE00041F7ED3211F4EF93F395F21718F43F93B8
:100BF000F395FBCF8F91B5DFFA95E1F70895E99171
:100C0000F9918591803021F0853219F0AADFF9CF72
:100C1000089520E0E89455915532C1F3503311F412
:100C2000689455915A3348F4505390F3220F022E92
:100C3000220F220F200D250FF4CF0EF4219589915C
:100C40009991533619F3533729F1533559F1BC01B2
:100C500088279927E8945C3621F4899199916894C2
:100C60005591543639F446EF7EF077FF0DC08FEF83
:100C70009FEF0AC055374AE039F0583540E121F07E
:100C8000523642E009F00895FF93EF937DDFEF9134
:100C9000FF91B7CFFF93EF93FC0181918030B9F3BF
:100CA00060DFFBCFFF93EF9368DFF1CFDF93CF934C
:100CB000CDB7DEB72596A3DFCF91DF910895282F1A
:100CC00080914101823071F08330B1F0813001F5C3
:100CD000E62FF0E038E0739FE00DF11D1124E2569D
:100CE000FC4F13C0E62FF0E088E0789FE00DF11D87
:100CF0001124E25EFC4F09C0E62FF0E038E0739F5C
:100D0000E00DF11D1124E256FD4FE491E03819F495
:100D100080E090E008959E2F9077892F90E034E056
:100D2000959587953A95E1F738E0239F800D911DC1
:100D3000112444E0880F991F4A95E1F7EF709C0158
:100D40002E0F311DF901EE0FFF1FE050F84985917C
:100D5000949108955998519A08955198599A0895DF
:100D60005898509A08955098589A08955198599AB9
:100D700085E08A95F1F7000089B186958170089524
:100D80005098589A85E08A95F1F7000089B18170F2
:100D90000895CF93DF93EC010E94B606882341F0BB
:100DA000209731F085E08A95F1F700002197F4CF84
:100DB000CE01DF91CF910895CF93DF93C2E3D0E0CE
:100DC0000E94B606811108C0209731F085E08A950F
:100DD000F1F700002197F4CFCE01DF91CF91089574
:100DE0002E9826982F9827980E94AA060E94B3064C
:100DF000E9E6F0E0808188608083E9980895E19ACF
:100E0000E99A0E94AD060C94B306E9980E94AA06DE
:100E10000C94B306CF93DF932FB7F894C0910201DF
:100E2000D0910301CE01882781159F4F19F080E0F2
:100E30009FEF02C08FEF90E08C2B9D2B90930301CE
:100E4000809302012FBFCE0199278F3F910581F535
:100E5000CD2FDD27C03FD10551F0CF3FD10509F49B
:100E600051C080917503C034D10599F407C08091B9
:100E7000750380FF33C08CE394E004C080FF2EC074
:100E800084E394E09F938F930E9456060F900F90F7
:100E900025C080FF37C0DF93CF938DE294E09F930E
:100EA0008F930E9456060F900F900F900F902AC0BC
:100EB000CE018F6F019699F08091750380FF0CC071
:100EC000DF93CF9385E294E09F938F930E94560621
:100ED0000F900F900F900F90CD2F01C0CFEF80910A
:100EE000750380FF0CC01F92CF938EE194E09F9317
:100EF0008F930E9456060F900F900F900F908C2F9B
:100F000090E002C08FEF9FEFDF91CF910895CF93D4
:100F1000CAE1C15069F00E940A078F3F2FEF920784
:100F200049F48FE99FE00197F1F700C00000F1CF8D
:100F30008FEF9FEFCF91089510923A0110923901EF
:100F4000109238011092370180E090E890930101EF
:100F5000809300018FEF9FEF909303018093020134
:100F60000895EF92FF920F931F93CF93DF93082F73
:100F7000109237018091750380FF0CC01F920F9370
:100F800082E494E09F938F930E9456060F900F90F7
:100F90000F900F90E9980E94AA060E94B3068FE86E
:100FA00091E00197F1F700C000000E94B0068FE8C1
:100FB00091E00197F1F700C000000E94AD0680E1CA
:100FC00097E20E94C906892B11F481E07FC0C0E03E
:100FD000D0E0FF24F39410E0EE24E39490E59A959A
:100FE000F1F7C8010C2E02C0959587950A94E2F797
:100FF00080FF04C0FE240E94B30602C00E94B00617
:101000000E94DC06892B11F482E060C082E390E04C
:101010000E94C906892B11F483E058C02196C8307C
:10102000D105E1F680E58A95F1F7FF2019F00E94DD
:10103000B30602C00E94B0060E94DC06892B11F4A0
:1010400084E044C082E390E00E94C906892B11F439
:1010500085E03CC090E59A95F1F70E94B3060E94A6
:10106000DC06892B11F486E031C082E390E00E9417
:10107000C906892B19F0C2E3D0E009C087E026C079
:10108000209759F025E02A95F1F7000021970E945A
:10109000C0068111F5CFCD2B11F488E017C00E9456
:1010A000DC06892B19F0C2E3D0E009C089E00EC04C
:1010B000209759F085E08A95F1F7000021970E946A
:1010C000C0068823A9F3CD2BB9F48AE080933701B9
:1010D000809137018061809337010E94AD060E94A4
:1010E000B306E19AE99A8FEF9FEFDF91CF911F91BD
:1010F0000F91FF90EF9008958FEF9FEF9093030172
:10110000809302010E949C070E94AD060E94B306D4
:10111000E19AE99ADF91CF911F910F91FF90EF90A3
:101120000C9487071F920F920FB60F9211242F93E2
:101130003F934F935F938F939F9329B18091760351
:1011400040910001509101014115504819F48093DC
:1011500036010FC090913601891B833050F0809189
:1011600000019091010190933A018093390180E24E
:10117000DDC0809100019091010196958795909333
:1011800001018093000120FF09C08091000190912E
:10119000010190689093010180930001809100010A
:1011A0009091010199278038910509F4F9C0A8F4BC
:1011B0008032910509F4F4C038F4009709F4F0C0C6
:1011C000409709F489C0A9C08034910509F4E8C0AA
:1011D0008035910509F480C0A0C0803C910539F1AB
:1011E00050F48039910509F477C0803A910509F0EF
:1011F00094C084E64DC0803D910509F46DC0803EE9
:10120000910509F08AC080910001909101019093AD
:101210003A01809339018091000190910101892F59
:101220009927909301018093000183E252C084E6E4
:1012300049990FC0882369F095E09A95F1F700006D
:101240008150F6CF882349F095E09A95F1F7000098
:1012500081504999F7CF8111A3C0809100019091ED
:10126000010190933A01809339018091000190919E
:101270000101892F9927909301018093000182E257
:1012800028C0882379F095E09A95F1F70000815005
:10129000499BF7CF07C0882349F095E09A95F1F76D
:1012A000000081504999F7CF81117AC080910001E7
:1012B0009091010190933A0180933901809100014E
:1012C00090910101892F992790930101809300014A
:1012D00081E28093380133C0809100019091010137
:1012E00090933A018093390180910001909101011E
:1012F00097FF02C080E101C081E1809338018091B5
:1013000000019091010146E0969587954A95E1F795
:10131000909301018093000112C08091000190918F
:10132000010190933A018093390180E8809337015D
:101330008091370190E0982F88278F6F27C0809188
:1013400000019091010199278F3F910511F480EFE1
:10135000EDCF809103018F3F31F0809102018F3FEB
:1013600011F080E4E3CF8091020190910301982F66
:10137000882790930301809302012091000130910E
:1013800001018091020190910301822B909303014E
:101390008093020180E090E8909301018093000126
:1013A0009F918F915F914F913F912F910F900FBE21
:1013B0000F901F901895CF93C82F8DEE0E94B10704
:1013C0008A3F910521F48C2FCF910C94B107CF91D6
:1013D0000895E82FE695E695E695EF70F0E0EB5B73
:1013E000FE4F4081282F277081E090E002C0880FD7
:1013F000991F2A95E2F7242F30E028233923232B45
:1014000011F4842B80830895E82FE695E695E69500
:10141000EF70F0E0EB5BFE4F2081382F377081E0FA
:1014200090E002C0880F991F3A95E2F7422F50E0F2
:1014300048235923452B19F08095822380830895F2
:10144000482F50E0FA013397E138F10508F048C021
:10145000E45BFF4F0C94242687E108958FE1089503
:101460008CE5089580E6089582E6089587E2089560
:1014700083E508958FE2089589E3089587E3089549
:101480008FE3089587E408958FE4089586E508952D
:101490008EE508958FE7089580E0089585E6089524
:1014A0008EE608958FE6089580E3089588E3089511
:1014B00080E4089588E4089580E5089587E5089517
:1014C0008FE5089588E1089588E0089580E2089501
:1014D00080E1089589E108958DE6089588E20895F0
:1014E0008F7708958FE00895CF93482F50E0FA0149
:1014F0007C97E834F105A0F5E353FF4F0C942426C4
:1015000085E53EC08AE53CC08BE53AC08CE538C035
:101510008DE536C08EE534C08FE532C080E630C040
:1015200081E62EC082E62CC083E62AC08FE628C062
:1015300081E726C082E724C084E722C085E720C077
:1015400087E71EC088E71CC08AE71AC08CE718C06E
:101550008FE716C080E714C089E712C08BE710C080
:10156000C82F1F928F938DE894E09F938F930E94D2
:1015700056060F900F900F900F908C2F01C084E5AE
:10158000CF9108950F931F93CF93DF930E94002470
:101590008C010E940A07EC01019631F4C8010E94F7
:1015A0001824843F9140A8F3CE01DF91CF911F9181
:1015B0000F9108950E94F0060C94FF068091750328
:1015C000816080937503E5E4F1E0119281E0E535F7
:1015D000F807D9F70895E82FF0E0EB5BFE4F808124
:1015E0000895E5E4F1E0119281E0E535F807D9F7D7
:1015F0000895982F80914101823048F092FB88270E
:1016000080F990FD826091FD84600C94DB0908955F
:10161000CF93DF9380913701882371F18091390155
:1016200090913A01209137019F938F931F922F93AE
:1016300087E195E09F938F930E9456068091370132
:1016400080750F900F900F900F900F900F9071F486
:10165000809140018B3051F480E195E09F938F930E
:101660000E945606109240010F900F901092370181
:1016700010923A011092390180913801882309F4BF
:1016800040C090913801809144019817D1F1809128
:10169000390190913A01209138019F938F931F92C5
:1016A0002F938CEF94E09F938F930E945606809126
:1016B00044010F900F900F900F900F900F9085FFA7
:1016C00004C09091380194FD06C084FF12C080913F
:1016D000380185FF0EC0809140018B3051F485EFB9
:1016E00094E09F938F930E945606109240010F90B2
:1016F0000F90809138018093440110923A0110922A
:101700003901E09140018E2F90E08C30910508F076
:1017100025C3FC01EB5EFE4F0C9424260E940507B6
:101720000E9400249F938F9380EF94E09F938F9368
:101730000E945606109241011092430110924201FC
:101740000E94F10A0E9482190E94002490933F0196
:1017500080933E0181E065C080913E0190913F0100
:101760000E941824893E934008F4F8C282E031C0F8
:101770000E949C070E94FF068FE99FE00197F1F706
:1017800000C000008FEF0E94B1078A3F910511F45D
:1017900086E001C083E0809340010E9400249F9373
:1017A0008F938BEE94E09F938F930E9456060F9039
:1017B0000F900F900F90D2C20E9405072E98269A84
:1017C0002F98279A0E94002490933F0180933E0116
:1017D00084E080934001C2C280913E0190913F011C
:1017E0000E941824853F914008F4B8C285E0F1CFEB
:1017F0002E9826982F9827980E949C070E94FF06F3
:101800000E9400249F938F9386EE94E09F938F9382
:101810000E9456060E94002490933F0180933E014F
:1018200086E080934001C3CF0E940A07019609F425
:1018300095C20E9400249F938F9381EE94E09F9322
:101840008F930E9456060E94002490933F0180933C
:101850003E0187E0E6CF80913E0190913F010E94DA
:101860001824853F914018F089E0809340010E9440
:101870000A07019609F472C20E9400249F938F9375
:101880008CED94E09F938F930E9456060E94002453
:1018900090933F0180933E0188E0C3CF80913E0149
:1018A00090913F010E941824853F914018F089E0F3
:1018B000809340010E940A07019609F44FC20E94DA
:1018C00000249F938F9387ED94E09F938F930E94C2
:1018D000560689E0A6CF82EF0E94B1078F3F2FEF17
:1018E000920789F08A3F910589F40E94C20A8F3FCE
:1018F0003FEF930771F0D82FCC270E94C20A9E01B8
:10190000282BC90108C08FEF9FEF05C08EEF9FEF16
:1019100002C080E090E090934301809342010E94D6
:1019200000249F938F9382ED94E09F938F930E9466
:10193000560680914201909143010F900F900F90B5
:101940000F90009711F482E02BC08F3F3FEF930779
:1019500011F481E025C08E3F2FEF9207A1F38F3F56
:10196000910559F48CEB94E09F938F930E94560657
:10197000109241010F900F901FC09C0125583B4AC7
:101980002230310580F480EF0E94B1078A3F910533
:10199000D1F683E00E94B1078A3F9105A1F683E06A
:1019A0008093410109C0803B3FEB9307C1F3882737
:1019B00081159F4BA1F3C7CF809141011F928F9357
:1019C000809143018F93809142018F938EEA94E03E
:1019D0009F938F930E9456068AE0809340010F9058
:1019E0000F900F900F900F900F90B8C10E9400249D
:1019F0009F938F9389EA94E09F938F930E9456065A
:101A00000F900F900F900F9080914101823029F03C
:101A1000833039F488EF0E94B1070E94FA160E94C1
:101A2000F90A8BE0809340010E9400249F938F93DA
:101A300084EA94E09F938F930E9456060F900F9034
:101A40000F900F900E940A079C012F3F9FEF3907CC
:101A500009F484C12115310519F02F3F310569F4CE
:101A60000E94F10A0E9482198CE994E09F938F935F
:101A70000E9456060F900F9071C1909141019230D3
:101A800009F44CC0933009F4CBC0913009F066C121
:101A900090913D01923099F028F4992341F09130D2
:101AA000C1F039C0933061F1943081F134C0803E8F
:101AB00021F0813E51F482E005C081E003C08D3108
:101AC000D9F483E080933D0149C187FFE3C08F775C
:101AD0000DC1863301F118F48A3229F41CC08A3A08
:101AE000D1F0863BC1F087FD03C00E94740A0BC091
:101AF0008F770E94740A0DC08D3969F484E0E2CFBB
:101B0000853449F485E50E94E90905C0853C19F44E
:101B100085E50E94040A10923D0120C1E0913C013C
:101B20004E2F50E04930510508F077C0FA01EF5DC3
:101B3000FE4F0C942426803E69F030F4833871F017
:101B4000843871F48FE757C0813E31F0803F41F413
:101B500081E05BC082E059C084E057C082E04BC0A6
:101B600087FF98C00E94F10A81E894E098C0893507
:101B700009F453C0803F19F0823119F44EC083E05C
:101B800044C010923C0187FD03C00E94200A82C01D
:101B90000E94F10A87E794E082C0833821F08438FC
:101BA00021F48FE738C082E036C010923C0187FFF5
:101BB0009DC00E94F10A8DE694E071C010923C0134
:101BC000823109F4CBC0893509F4C8C087FD03C050
:101BD0000E94200A8BC00E94F10A80E694E05FC058
:101BE000843121F0803FC9F486E00FC085E00DC04C
:101BF000873799F480E00E94E9090FC0843169F4C5
:101C000087E003C0803F49F488E080933C01A6C090
:101C1000873719F480E00E94040A10923C019EC0AC
:101C200090913B01913009F443C038F0923009F4AF
:101C300063C0933009F47FC091C0863809F168F41D
:101C40008338D1F020F4803819F582E06CC08438F4
:101C5000A9F08538E9F48BE01DC08C38A9F030F488
:101C6000873881F08B38A1F481E014C08D3871F091
:101C7000803F71F481E057C082E00CC08FE70AC05A
:101C800086E008C080E006C089E004C08AE002C0A7
:101C900087FD03C00E94E90961C083E594E09F933A
:101CA0008F930E9456060F900F901092400156C0DD
:101CB000482F50E0FA01E358F109EB30F10590F4B8
:101CC000E65DFE4F0C94242682E045C08FE743C0BA
:101CD0008BE041C086E03FC081E03DC089E03BC071
:101CE0008AE039C010923B0187FD03C00E94040ABC
:101CF00035C089E494E0D3CF853279F030F4863171
:101D000071F08E3199F480E00BC0863221F0803F73
:101D100069F483E008C08DE503C083E501C081E577
:101D20000E94E90905C080933B0118C00E94F10A96
:101D300010923B0113C08E3169F020F48631B1F767
:101D400081E509C0853221F0863281F78DE503C037
:101D500083E501C080E00E94040AEACF81E0DF91C0
:101D6000CF9108958091790208950895CF93DF93DC
:101D700000D01F92CDB7DEB720917F03243021F52C
:101D800023E029839B838A8382E08093E9008FEF9D
:101D90009091E800815095FD06C095ED9A95F1F778
:101DA00000008111F5CF8091E80085FF0DC040E073
:101DB00050E063E070E0CE0101960E942213809112
:101DC000E8008E778093E8000F900F900F90DF91DE
:101DD000CF910895CF93DF9300D01F92CDB7DEB798
:101DE00020917F03243029F522E02983805891092E
:101DF0009B838A832093E9008FEF9091E8008150C4
:101E000095FD06C095ED9A95F1F700008111F5CF8B
:101E10008091E80085FF0DC040E050E063E070E095
:101E2000CE0101960E9422138091E8008E77809364
:101E3000E8000F900F900F90DF91CF910895CF930E
:101E4000DF93EC0190917F03943009F048C08091BA
:101E500014018823D9F0809115018823B9F090935B
:101E6000E90081E8815049F09091E80095FD05C0B6
:101E70009AE29A95F1F700C0F5CF8091E80085FFCE
:101E80002EC040E050E060E270E019C081E0809335
:101E9000E90081E8815059F09091E80095FD07C074
:101EA000EFE3F1E03197F1F700C00000F3CF80914C
:101EB000E80085FF14C040E050E068E070E0CE012B
:101EC0000E9422138091E8008E778093E80080E2E0
:101ED000FE01A9E5B2E001900D928A95E1F7DF914C
:101EE000CF910895CF93C0915701C1110BC00E94AB
:101EF0000C24643C79408105910520F081E08093B9
:101F00005701C1E08C2FCF910895FF920F931F933B
:101F1000CF93DF93D82F0FB607FE83C080917F0346
:101F2000843081F08091070190E0019620910901B1
:101F300030E0822393232091080130E08217930739
:101F400009F0CBC00E94720F811110C0809107016F
:101F500090E001962091090130E0822393232091A3
:101F6000080130E08217930709F0B7C00E940024EF
:101F70008C01C091E900CF709091EC00892F8170A5
:101F800090FD80E8C82B83E08093E90085E0F82E7F
:101F90008091EB0085FD42C08091EB0080FF3EC048
:101FA0008091EE0087FF3AC080910801909107016F
:101FB000981709F457C09091E80095FF8CC0E09104
:101FC0000501F0910601E80FF11D20818F5F9091CE
:101FD00009018923809308012093F1008091E80092
:101FE00085FDE2CF8091E80080FFDECF8091E800A0
:101FF0008E778093E800F0920401D6CF809107019C
:1020000090E001962091090130E0822393232091F2
:10201000080130E08217930709F44AC0CF70C093DB
:10202000E90040910701842F90E001962091090179
:1020300030E0822393232091080130E08217930738
:1020400009F44EC0E0910501F0910601E40FF11D85
:10205000D083809107018F5F90910901892380933C
:1020600007013EC08091E80085FF35C0D093F100A4
:1020700081E02091F2003091F300232B91F09091B8
:10208000E80090FF0EC09091E80095FF03C0109209
:10209000F100F9CF9091E8009E779093E800F092DC
:1020A0000401882309F4AACFCF70C093E90018C0B7
:1020B00080910401882309F4B1CF0E9400249C017F
:1020C0008017910711F4890163CF90910401915019
:1020D00090930401F8CF80E0CCCF40910701B2CFBC
:1020E00080E0DF91CF911F910F91FF900895809133
:1020F0007E03811104C00E948A150C94EC1508958A
:1021000010927E030895089542E061EC81E00E9400
:102110009B1242E061EC82E00E949B1242E261EC81
:1021200083E00E949B1242E261EC84E00C949B12DB
:1021300080918103833009F455C030F4813071F00F
:10214000823009F48EC008958A3009F47AC08B3049
:1021500009F460C0893009F09CC020C080918003E0
:10216000813A09F096C08091E800877F8093E8006B
:102170008091840390918503892B21F460E289E5A5
:1021800092E003C060E080E090E070E00E946F1396
:102190008091E8008B778093E80008958091800318
:1021A000813209F076C08091840390918503009775
:1021B00019F0039709F06DC08091E800877F809344
:1021C000E8008091E80082FD05C080917F038111C5
:1021D000F8CF5FC08091F100809379028091E80090
:1021E0008B7753C080918003813A09F052C080916F
:1021F000840390918503892B09F04BC08091E800FE
:10220000877F8093E8008091E80080FFFCCF809179
:10221000140136C0809180038132D9F58091840306
:1022200090918503892BA9F58091E800877F8093A1
:10223000E8000E94D01280918203809314010C94D4
:10224000821980918003813221F58091E800877F97
:102250008093E8000E94D0128091830380937A02D9
:10226000089580918003813AA1F48091E800877FEE
:102270008093E8008091E80080FFFCCF80917A0293
:102280008093F1008091E8008E778093E8000C94B1
:10229000D0120895809179028093580110927902AA
:1022A0000E94F10A0C9482190C944A110E94AD23E9
:1022B00080917D03882329F00E94BA2381110C9418
:1022C000851208950E94CE2380915801809379024F
:1022D00008950C94621108950C946B11CF9384B7F8
:1022E000877F84BF0FB6F894A895809160008861BD
:1022F00080936000109260000FBE90E080E80FB6FF
:10230000F89480936100909361000FBE85E89FE090
:102310000E9480238AE091E00E94F5168FE495E008
:102320000E94BD050E94DA0A0E94A9170E948A1520
:102330000E94EC1578940E94AB1780917F03843043
:1023400029F00E94DA160E946B11F7CF8DE395E019
:102350000E94BD050E946C118BE295E00E94BD05B4
:10236000C3E080917F03853019F40E945611F9CFA4
:102370000E94AF172091E4003091E5008091550153
:10238000909156012817390709F466C08091E4003E
:102390009091E50090935601809355010E94720F31
:1023A000882309F459C080917F03843009F054C018
:1023B0008091E9008F702091EC00922F917020FDA8
:1023C00090E8892BC093E9009091EB0090FF41C009
:1023D0009091EE0097FF3DC0909108012091070178
:1023E000291709F12091E80025FF1DC0E0910501A2
:1023F000F0910601E90FF11D30819F5F20910901E5
:102400009223909308013093F1009091E80095FD9C
:10241000E3CF9091E80090FFDFCF9091E8009E77A6
:102420009093E800D9CF2091F2003091F300232B54
:1024300081F09091E80090FF0CC09091E80095FF2A
:1024400003C01092F100F9CF9091E8009E7790932D
:10245000E8008F708093E9000E94DA1682CF292F5E
:10246000332723303105C9F060F42130310581F084
:102470002230310509F041C084E790E02FEA35E0D1
:1024800040C021323105E1F02232310531F135C051
:1024900082E190E023E236E034C099278130910553
:1024A00049F028F0029749F5E5E6F5E005C0EBEACA
:1024B000F5E002C0EBE9F5E0849190E09F0121C0D6
:1024C00064307105D0F4660F771FFB01EC5DFE4FA1
:1024D0002081318189E090E014C06430710568F496
:1024E000FB01EE0FFF1FE45EFE4F20813181FB01F7
:1024F000E85EFE4F808190E004C080E090E020E044
:1025000030E0FA0131832083089584E189BD86E1BA
:1025100089BD09B400FEFDCF8091D8008F7D8093E6
:10252000D8008091E00082608093E0008091E0001C
:1025300081FDFCCF0895982F973068F59093E900BE
:10254000981739F07091EC002091ED005091F00057
:1025500003C0242F762F50E021FD02C09F5FECCFF7
:102560003091EB003E7F3093EB003091ED003D7FEA
:102570003093ED003091EB0031603093EB007093BD
:10258000EC002093ED005093F0002091EE0027FD29
:10259000E5CF80E008958F708093E90081E0089591
:1025A0008091800387FF11C08091E80082FD05C003
:1025B00080917F038111F8CF11C08091E8008B7763
:1025C0000BC080917F03882349F08091E80080FF51
:1025D000F8CF8091E8008E778093E80008952091ED
:1025E000E4003091E50095E64091EC00842F817085
:1025F00040FF23C08091E80080FD1DC080917F03D3
:10260000882399F0853099F08091EB0085FD11C009
:102610004091E4005091E5002417350729F39150CB
:1026200011F09A01E1CF84E0089582E0089583E0FB
:10263000089581E0089580E008954091E80042FF08
:10264000DDCF0895CF92DF92EF92FF920F931F9309
:10265000CF93DF93EC018B017A010E94EF1281117D
:1026600035C0E114F10439F0F70180819181081B34
:10267000190BC80FD91FC12CD12C0115110529F137
:102680008091E80085FD18C08091E8008E778093E6
:10269000E8000E94DA16E114F10449F0F7018081A4
:1026A0009181C80ED91ED182C08285E00FC00E94E0
:1026B000EF12882311F30AC089918093F100015031
:1026C0001109FFEFCF1ADF0AD8CF80E0DF91CF9159
:1026D0001F910F91FF90EF90DF90CF900895209180
:1026E0008603309187032617370748F06115710577
:1026F00039F42091E8002E772093E80001C0B90159
:10270000FC0120E06115710569F180917F03882348
:10271000E1F18530E1F18091E80083FD3AC08091DC
:10272000E80082FD2CC08091E80080FFEBCF809113
:10273000F2009091F3006115710551F08830910518
:1027400038F421912093F100615071090196F3CF83
:1027500021E0089709F020E08091E8008E778093CF
:10276000E800D0CF2111D1CF0AC080917F03882308
:1027700061F0853061F08091E80083FD0AC08091AE
:10278000E80082FFF2CF80E0089582E0089583E0C0
:10279000089581E0089520918603309187032617DC
:1027A000370748F06115710539F42091E8002E775C
:1027B0002093E80001C0B901FC0120E0611571051A
:1027C00081F180917F03882309F43EC0853009F4AC
:1027D0003DC08091E80083FD3BC08091E80082FD10
:1027E0002DC08091E80080FFE9CF8091F2009091A8
:1027F000F3006115710559F08830910540F424917A
:102800002093F1003196615071090196F2CF21E0D9
:10281000089709F020E08091E8008E778093E80027
:10282000CDCF2111CECF0AC080917F03882361F0E4
:10283000853061F08091E80083FD0AC08091E80056
:1028400082FFF2CF80E0089582E0089583E008954A
:1028500081E008951F93CF93DF93CDB7DEB7AA979A
:102860000FB6F894DEBF0FBECDBFE0E8F3E0809175
:10287000F100819323E0E838F207C9F70E9498102D
:102880008091E80083FF2EC18091800390918103A5
:10289000492F50E04A30510508F024C1FA01EB5CA1
:1028A000FE4F0C942426803821F0823809F01AC19A
:1028B00008C080917C0390917D03992389F0826008
:1028C0000FC0809184038F70873008F00BC1809314
:1028D000E9008091EB0085FB882780F91092E900E0
:1028E0009091E800977F9093E8008093F100109218
:1028F000F100D1C0282F2D7F09F0F4C0882319F0F2
:10290000823061F0EFC080918203813009F0EAC02B
:10291000933009F080E080937D032EC08091820384
:1029200081112AC0809184038F702FEF280F2630E9
:1029300008F0D8C08093E9002091EB0020FF1CC074
:10294000933021F48091EB00806214C09091EB00F1
:1029500090619093EB0021E030E0A90102C0440FA8
:10296000551F8A95E2F74093EA001092EA008091A1
:10297000EB0088608093EB001092E9008091E80002
:10298000877F8093E8000E94D012ACC08111AAC05A
:10299000109182031F778091E3008078812B8093D0
:1029A000E3008091E800877F8093E8000E94D012C6
:1029B0008091E80080FFFCCF8091E30080688093E5
:1029C000E300111102C082E001C083E080937F0325
:1029D00089C08058823008F085C080918203909130
:1029E00083038C3D53E0950779F583E08A838AE27F
:1029F00089834FB7F894DE01139620E03EE051E260
:102A0000E32FF0E050935700E49120FF03C0E295DC
:102A1000EF703F5FEF708E2F90E0EA3010F0C796B6
:102A200001C0C0968D939D932F5F243149F74FBF0E
:102A30008091E800877F8093E8006AE270E0CE0131
:102A400001960E946F1316C06091840370918503F4
:102A5000AE014F5F5F4F0E942F12BC01892B09F41A
:102A600041C09091E800977F9093E80089819A8116
:102A70000E94CB138091E8008B778093E80032C0EE
:102A8000803881F58091E800877F8093E80080910D
:102A90007B038093F1008091E8008E7772CF8111E3
:102AA00021C0809182039091830399270297D4F4E7
:102AB0008091E800877F8093E80080918203809373
:102AC0007B030E94D01280917B03811106C080910C
:102AD000E30087FD02C081E001C084E080937F03B2
:102AE0000E9484108091E80083FF0AC08091E80072
:102AF000877F8093E8008091EB0080628093EB00F9
:102B0000AA960FB6F894DEBF0FBECDBFDF91CF916E
:102B10001F9108950E94FB150E940316E0EEF0E05D
:102B2000808181608083E8EDF0E080818F77808311
:102B300019BCA7EDB0E08C918E7F8C9380818F7E45
:102B4000808310927E0308950F931F93CF93DF939A
:102B50000E94FB150E940316C8EDD0E088818F7794
:102B6000888388818068888388818F7D8883E7ED6A
:102B7000F0E080818068808319BC10927F031092FE
:102B80007B0310927D0310927C0300EE10E0F801AD
:102B900080818B7F808388818160888342E060E0D0
:102BA00080E00E949B12E1EEF0E080818E7F8083C6
:102BB000E2EEF0E0808181608083808188608083A4
:102BC000F80180818E7F8083888180618883DF9196
:102BD000CF911F910F910895E8EDF0E080818F7EF5
:102BE0008083E7EDF0E080818160808381E08093E5
:102BF0007E030C94A415E8EDF0E080818C7F808347
:102C00001092E20008951092DA001092E100089507
:102C10001F920F920FB60F9211240BB60F922F93A3
:102C20003F934F935F936F937F938F939F93AF9354
:102C3000BF93EF93FF938091E10082FF0BC08091DF
:102C4000E20082FF07C08091E1008B7F8093E1006A
:102C50000E94D9168091DA0080FF1FC08091D800B1
:102C600080FF1BC08091DA008E7F8093DA00809114
:102C7000D90080FF0DC084E189BD86E189BD09B41A
:102C800000FEFDCF81E080937F030E94771005C096
:102C900019BC10927F030E9480108091E10080FF98
:102CA00019C08091E20080FF15C08091E2008E7F04
:102CB0008093E2008091E20080618093E200809145
:102CC000D80080628093D80019BC85E080937F0390
:102CD0000E9454118091E10084FF30C08091E20095
:102CE00084FF2CC084E189BD86E189BD09B400FE62
:102CF000FDCF8091D8008F7D8093D8008091E10036
:102D00008F7E8093E1008091E2008F7E8093E200CD
:102D10008091E20081608093E20080917B038823B0
:102D200011F084E007C08091E30087FD02C081E0DC
:102D300001C083E080937F030E9469118091E100CC
:102D400083FF24C08091E20083FF20C08091E100D6
:102D5000877F8093E10082E080937F0310927B0362
:102D60008091E1008E7F8093E1008091E2008E7F70
:102D70008093E2008091E20080618093E20042E073
:102D800060E080E00E949B120E948310FF91EF910F
:102D9000BF91AF919F918F917F916F915F914F9173
:102DA0003F912F910F900BBE0F900FBE0F901F9071
:102DB00018950895CF9380917F038823A1F0C09147
:102DC000E900CF709091EC00892F817090FD80E830
:102DD000C82B1092E9008091E80083FD0E942A141C
:102DE000CF70C093E900CF910895909380028093B3
:102DF0007F020895E0917F02F0918002309721F0E8
:102E00000190F081E02D099480E00895EF92FF9207
:102E10000F931F93CF93DF93E0917F02F091800295
:102E20003097B1F18C010280F381E02D09958091FA
:102E3000750382FF2DC080FF04C08CE297E00E94E2
:102E4000BD05E80110E286E2E82E87E0F82E8091C9
:102E5000750380FF0BC088811F928F93FF92EF92C2
:102E60000E9456060F900F900F900F9011502196D0
:102E70001111EDCF8091750380FF0AC084E297E0C5
:102E8000DF91CF911F910F91FF90EF900C94BD05B2
:102E9000DF91CF911F910F91FF90EF900895CF9305
:102EA000DF9320917D0230917E022817390709F1C6
:102EB00090937E0280937D02E0917F02F0918002E8
:102EC0003097B9F0EC010680F781E02D09958091EB
:102ED000750382FF0EC080FF0CC0DF93CF9386E1A5
:102EE00097E09F938F930E9456060F900F900F903C
:102EF0000F90DF91CF910895CF93DF9320917B02C4
:102F000030917C022817390709F190937C02809355
:102F10007B02E0917F02F09180023097B9F0EC01E2
:102F20000084F185E02D09958091750382FF0EC024
:102F300080FF0CC0DF93CF9386E097E09F938F9341
:102F40000E9456060F900F900F900F90DF91CF9137
:102F500008950C9452180E94F7230C94DE0ABF9235
:102F6000CF92DF92EF92FF920F931F93CF93DF9355
:102F700000D000D01F92CDB7DEB70E94080B02E848
:102F800012E0F12C8F2D0E94EB0AB82EF801C080C0
:102F9000C82639F4F3940F5F1F4FF0E1FF12F2CF10
:102FA00030C08091750381FD0E945318D12CEE240E
:102FB000E3948C2D8E21F9F0D982FA8291E08B2D49
:102FC0008E2109F490E09B830E9400248160782F79
:102FD0009D838C8349815A816B818D810E948918E0
:102FE00049815A816B817C818D810E949823F801EF
:102FF00080818E258083D394EE0CF8E0DF12D9CF48
:10300000C9CF8FEF89838A831B820E94002481604D
:10301000782F9D838C8349815A816B818D810E9499
:1030200089180E9497230E94FA16909181028917AD
:1030300041F10E94FA16809381029091750392FFEC
:103040000EC090FF0CC01F928F9387E397E09F9371
:103050008F930E9456060F900F900F900F908091C3
:1030600081020F900F900F900F900F90DF91CF91F2
:103070001F910F91FF90EF90DF90CF90BF900C9435
:10308000A9230F900F900F900F900F90DF91CF9189
:103090001F910F91FF90EF90DF90CF90BF90089518
:1030A0000C94F90A0895EF92FF920F931F93CF9318
:1030B000DF938DE497E00E94BD05C0E0D0E08CE294
:1030C000E82E81E0F82E02E417E08C2F0E94EB0A34
:1030D0000E948523FF92EF921F928F93DF93CF93ED
:1030E0001F930F930E94560621968DB79EB70896A0
:1030F0000FB6F8949EBF0FBE8DBFC031D10529F722
:10310000DF91CF911F910F91FF90EF900895089557
:103110000895CF93DF93CDB7DEB72B970FB6F89412
:10312000DEBF0FBECDBF942F4F83252F58876987F1
:103130007A878B874A855B85452B31F02F3F31F4A9
:1031400081E09F3F19F403C081E001C080E080FD71
:1031500007C04F81588569857A858B850E949823A1
:10316000DE01119686E0FD0111928A95E9F785E06E
:10317000FE01379601900D928A95E1F749815A81B7
:103180006B817C818D819E810E94931F2B960FB64F
:10319000F894DEBF0FBECDBFDF91CF910895CF93DE
:1031A000882309F465C0C82F8CEF8C0F813A20F07A
:1031B00080E58C0F8E3248F48C2F0E94D12581112E
:1031C00057C08C2F0E947B220CC080E28C0F88306D
:1031D00058F4C77081E001C0880FCA95EAF70E94D1
:1031E0002023CF910C945A238BE58C0F833078F4F5
:1031F000C53A29F0C63A31F083E890E005C081E88D
:1032000090E002C082E890E0CF910C944F1788E5DF
:103210008C0F873168F5C83A89F0C93A91F0CA3AFB
:1032200099F0CB3AA1F0CC3AA9F0CD3AB1F0CE3A30
:10323000B9F0CF3AC1F080E090E017C082EE90E0A4
:1032400014C089EE90E011C08AEE90E00EC085EBCC
:1032500090E00BC086EB90E008C083EB90E005C0E7
:1032600084EB90E002C087EB90E0CF910C947C1748
:10327000CF910895882349F19CEF980F913A20F05F
:1032800090E5980F9E3218F40E94CB220DC090E278
:10329000980F983058F4877091E001C0990F8A9583
:1032A000EAF7892F0E9426230C945A239BE5980F56
:1032B000933020F480E090E00C944F17885A8731C7
:1032C00020F480E090E00C947C170895882321F08E
:1032D0000E9420230C945A230895882321F00E94F1
:1032E00026230C945A2308950E9440230E940F2302
:1032F0000E945A2380E090E00E944F1780E090E007
:103300000C947C170E9430230C947419CF92DF9296
:10331000EF92FF920F931F93CF93DF9300D000D0D3
:103320001F92CDB7DEB76C010E94AB23811101C3A0
:1033300085E0F601DE01119601900D928A95E1F784
:10334000F60140815181238134812115310531F00D
:103350005F3F31F481E04F3F19F403C081E001C0C9
:1033600080E080FDE6C2F601F280E580E2948FE025
:10337000E82249835A83FB82722F3D832C836F2D71
:103380008D810E94F7218C010E94F6210E94E62087
:10339000E12FE295EF708E2F90E0FC01E15CFE4F93
:1033A0000C942426812F807F1F70882311F01295A2
:1033B000107FFF20B9F0112329F0812F0E943323C1
:1033C0000E945A23802F0F900F900F900F900F9014
:1033D000DF91CF911F910F91FF90EF90DF90CF90F1
:1033E0000C94CF18802F0E943A19112309F4A1C21E
:1033F000812F0E9439230F900F900F900F900F9004
:10340000DF91CF911F910F91FF90EF90DF90CF90C0
:103410000C945A23812F807F1F70803211F01295F7
:10342000107F002319F0013009F12BC0FF20A9F013
:10343000EE2059F1F1E0812FEF1228C00F900F908C
:103440000F900F900F90DF91CF911F910F91FF90F0
:10345000EF90DF90CF900C944323EE2021F021E0F9
:10346000E21609F466C20E9446234DC0FF20E9F02F
:1034700085E08E1508F45DC20E941D23812329F08A
:1034800042C0FF20F1F1E11015C0812F0F900F9085
:103490000F900F900F90DF91CF911F910F91FF90A0
:1034A000EF90DF90CF900C94661994E09E1508F48D
:1034B00040C229C0F601858180FF13C08F708583CB
:1034C000E4CF003F09F472C108F03EC180E4800FF0
:1034D000803208F442C1FF2009F4D3C1EE2009F480
:1034E00083C1802F0E94CF18093309F0C3C1FFEFB9
:1034F00021EE84E0F15020408040E1F700C0000060
:1035000018C2E110C0C1812F42C1812F86958695D6
:10351000837019F08130B9F00CC2FF2019F0C80196
:10352000937002C080E090E00F900F900F900F908A
:103530000F90DF91CF911F910F91FF90EF90DF904F
:10354000CF900C944F17FF2019F0C801937002C060
:1035500080E090E00F900F900F900F900F90DF9110
:10356000CF911F910F91FF90EF90DF90CF900C942F
:103570007C17812F837009F070C0F110DAC1202F01
:10358000229526952770220F220F602F6F70862FAD
:1035900090E0A0E0B0E06C017D01022E04C0CC0CF4
:1035A000DD1CEE1CFF1C0A94D2F704FF12C08FE052
:1035B00090E0A0E0B0E004C0880F991FAA1FBB1FD5
:1035C0002A95D2F7BC01CD016095709580959095B4
:1035D00003C060E070E0CB011695169513701230B1
:1035E000B1F040F56C297D298E299F29113031F1E8
:1035F0000F900F900F900F900F90DF91CF911F9130
:103600000F91FF90EF90DF90CF900C940B216C29DD
:103610007D298E299F290F900F900F900F900F906A
:10362000DF91CF911F910F91FF90EF90DF90CF909E
:103630000C9425210E940B21C701B6010F900F9019
:103640000F900F900F90DF91CF911F910F91FF90EE
:10365000EF90DF90CF900C94F120FF2019F0812F94
:10366000817001C08695882309F463C1202F2295BB
:1036700026952770220F220F602F6F70862F90E003
:10368000A0E0B0E06C017D01022E04C0CC0CDD1C7A
:10369000EE1CFF1C0A94D2F704FF12C08FE090E0EA
:1036A000A0E0B0E004C0880F991FAA1FBB1F2A9595
:1036B000D2F7BC01CD01609570958095909503C0BF
:1036C00060E070E0CB011695169513701230B1F0E2
:1036D00040F56C297D298E299F29113031F10F90F9
:1036E0000F900F900F900F90DF91CF911F910F913E
:1036F000FF90EF90DF90CF900C94D2216C297D2920
:103700008E299F290F900F900F900F900F90DF91AF
:10371000CF911F910F91FF90EF90DF90CF900C947D
:10372000E4210E94D221C701B6010F900F900F90A3
:103730000F900F90DF91CF911F910F91FF90EF901D
:10374000DF90CF900C94C021023F09F45EC008F4D2
:1037500049C0033F09F46CC0BECE902F9071E92E92
:10376000812F8F71FF2051F00E945921802FEE2070
:1037700019F08295807F8ACE8F7088CE0E947A2140
:10378000802FEE2019F08295807F01C08F700F90FE
:103790000F900F900F900F90DF91CF911F910F918D
:1037A000FF90EF90DF90CF900C946D19FF20A9F05F
:1037B000E4E0EE1508F4BDC0812F8F710F900F90DB
:1037C0000F900F900F90DF91CF911F910F91FF906D
:1037D000EF90DF90CF900C949F21F5E0FE1508F458
:1037E000A8C0EACFFF2099F0812F8F710F900F9022
:1037F0000F900F900F90DF91CF911F910F91FF903D
:10380000EF90DF90CF900C945921FF2069F3812F26
:103810008F710F900F900F900F900F90DF91CF91BD
:103820001F910F91FF90EF90DF90CF900C947A2131
:10383000FF2089F0812F8F710F900F900F900F90C4
:103840000F90DF91CF911F910F91FF90EF90DF903C
:10385000CF900C9444210F900F900F900F900F90E9
:10386000DF91CF911F910F91FF90EF90DF90CF905C
:103870000C943F21033509F43ACE073409F059C0BE
:1038800036CEEE2021F2802F0F900F900F900F90E8
:103890000F90DF91CF911F910F91FF90EF90DF90EC
:1038A000CF900C943A19412F4F70602FC6010E949F
:1038B0006C240F900F900F900F900F90DF91CF918D
:1038C0001F910F91FF90EF90DF90CF900C944120CB
:1038D00001112FC0FF2069F10E9482192FEF80E7AC
:1038E00092E0215080409040E1F700C000000F902E
:1038F0000F900F900F900F90DF91CF911F910F912C
:10390000FF90EF90DF90CF900C944D24412F4F709B
:10391000602FC6010F900F900F900F900F90DF91C6
:10392000CF911F910F91FF90EF90DF90CF900C946B
:103930006F240F900F900F900F900F90DF91CF9109
:103940001F910F91FF90EF90DF90CF9008951F93FC
:10395000CF93DF9300D000D01F92CDB7DEB7942F66
:103960004983252F5A836B837C838D834C815D81B2
:10397000452B31F02F3F31F481E09F3F19F403C014
:1039800081E001C080E0182F117080FD31C04981B5
:103990005A816B817C818D810E94F721292F22958C
:1039A0002F702C3030F42A30A0F42250223030F026
:1039B00022C02C30C9F02F30B9F01DC0853A28F450
:1039C0008430C0F4823028F415C090E2980F98300B
:1039D00088F0883E30F4803E68F48450813A58F490
:1039E00009C0803F41F406C093FB112710F903C0C2
:1039F00010E001C011E0812F0F900F900F900F90F9
:103A00000F90DF91CF911F910895CF93DF9300D056
:103A100000D01F92CDB7DEB70F900F900F900F9090
:103A20000F90DF91CF910895CF93DF9300D000D016
:103A300000D0CDB7DEB726960FB6F894DEBF0FBE26
:103A4000CDBFDF91CF9108951F93CF93DF93C091A6
:103A5000920216E080919302C81799F0D0E01C9F63
:103A6000F0011D9FF00D1124EC56FD4F4081518156
:103A700062817381848195810E94141D2196C77093
:103A8000E9CFDF91CF911F9108954091C4025091E9
:103A9000C5026091C6027091C7028091C8029091E0
:103AA000C9020C94141D0F931F93CF93DF93809141
:103AB000C90282958F7009F05DC08091C60288238B
:103AC00009F458C080919202109193026091C4024F
:103AD0007091C502C091C702D091C80291E06F3FBA
:103AE00009F090E0292F06E0811709F443C02097E0
:103AF00021F07F3F21F030E003C031E001C0322FE0
:103B000090E030FD34C0089FF001099FF00D1124B2
:103B1000DF01AC56BD4F11963C911197371327C06A
:103B20003C91361324C012963C91129731111FC05C
:103B300013964D915C9114974C1B5D0B483C5105BD
:103B4000B0F48091C9028F7080618093C902E756FA
:103B5000FD4F80818F708061808384EC92E00E94B1
:103B60008619DF91CF911F910F910C94241D01961E
:103B70008770BACFDF91CF911F910F9108959F92D7
:103B8000AF92BF92CF92DF92EF92FF920F931F936B
:103B9000CF93DF93CDB7DEB761970FB6F894DEBF52
:103BA0000FBECDBF8C0185E0F801DE011D960190AE
:103BB0000D928A95E1F7F80140815181F280C3802E
:103BC000D4809091C4026091C5022091C7023091C7
:103BD000C8022115310531F06F3F31F481E09F3F7C
:103BE00019F403C081E001C080E0F82FF1709F2E2E
:103BF00080FD52C184ECA82E82E0B82EE090C6026F
:103C0000F601E21BF30BEE2009F4E8C08091C90233
:103C1000E83CF10508F0A4C0282F207F09F053C02C
:103C2000561313C0491311C0EF2CF1100EC08F7042
:103C300080618093C9020E94451DC5010E948619BA
:103C40008091C902F80185835BC1C114D10431F0B0
:103C50005F3F31F481E04F3F19F403C081E001C0C0
:103C600080E080FD03C081E08F2502C080E090E00D
:103C7000F82FF170EF2E80FF1CC0809192022091EE
:103C8000930236E0821709F418C190E0389FF001E2
:103C9000399FF00D1124EC56FD4F6181561306C07B
:103CA0006081461303C06281F61203C001968770DB
:103CB000E9CFEF2CFF2009F423C18091C902816074
:103CC0008093C90262C0561306C0491304C0F110A4
:103CD00002C0F801A7C04D875E87FF867C2DD98A78
:103CE000C88A6F2D89890E94A71C882399F1FF201B
:103CF00089F12091C902822F82958F7090E00297FE
:103D000074F08091C4029091C50298878F831986C0
:103D1000DB86CA862C87CE0107960E94861986E02C
:103D2000F801A4ECB2E001900D928A95E1F70E94AF
:103D3000531D0E94451D11C0561749F14D875E87DE
:103D4000FF867C2DD98AC88A6F2D89890E94A71C7D
:103D500081112CC0C8010E948619EE24E394D0C0C2
:103D6000282F207F49F77C2DD98AC88A6F2D898911
:103D70000E94051D84EC92E00E94861986E0F50100
:103D800011928A95E9F70E94451DE12CB9C04913AB
:103D9000D5CFF110D3CFF8018583C8010E948619D1
:103DA00086E0F50111928A95E9F7AAC0FF2091F209
:103DB0002091C902822F82958F7090E002970CF4B7
:103DC000AECF8091C4029091C5029A8389831B82F1
:103DD000DD82CC822E83CE0101969FCFE83CF10597
:103DE00008F04BC0EF2CFF2009F4B4CF561330C0BD
:103DF00049132EC02091C90220FD21C0822F829537
:103E00008F70482F50E041155105C9F0F801258306
:103E10004F30510541F08F5F982F9295907F822F00
:103E20008F70892B8583C8010E94861986E0F8016E
:103E3000A4ECB2E001900D928A95E1F72AC086E0E9
:103E4000F801A4ECB2E001900D928A95E1F758C018
:103E50004D875E87FF867C2DD98AC88A6F2D898918
:103E60000E94A71C81115BCF8091C9028160809361
:103E7000C902C8010E94861943C07C2DD98AC88A0C
:103E80006F2D89890E94051D86E0F50111928A95A2
:103E9000E9F70E94451D34C0FF2009F45BCF4D8730
:103EA0005E87FF867C2DD98AC88A6F2D89890E94FA
:103EB000A71C882309F44ECF32CF7C2DD98AC88A1B
:103EC0006F2D89890E94F721292F22952F7022308A
:103ED00028F49F7039F0811105C00BC0243028F4FC
:103EE0009F7049F4805E883020F0C8010E948619D6
:103EF0009E2CE92C05C0F8019581907F99F7F9CFA8
:103F00008E2D61960FB6F894DEBF0FBECDBFDF9148
:103F1000CF911F910F91FF90EF90DF90CF90BF90C6
:103F2000AF909F9008951F93CF93DF93CDB7DEB7E7
:103F30002C970FB6F894DEBF0FBECDBF4F835887C6
:103F400069877A878B879C87CE0107960E94BF1D61
:103F50008823D1F09F8188852A853B85232B31F0EA
:103F60008F3F31F481E09F3F19F403C081E001C02D
:103F700080E080FD47C04F81588569857A858B85B3
:103F80009C850E94141D3EC086E0FE013796DE012E
:103F9000119601900D928A95E1F7FF81E8856A8577
:103FA0007B856115710531F0EF3F31F481E0FF3F12
:103FB00019F403C081E001C080E080FD23C020919E
:103FC000930230E0C90101968770992740919202CF
:103FD00050E084179507F1F1F983EA837D836C83C0
:103FE00096E0929FD001939FB00D1124AC56BD4F27
:103FF000FE01319601900D929A95E1F7809393021C
:104000000E94241D16E080919202909193028917DC
:1040100071F1189FC00111248C569D4F0E94BF1D45
:10402000882329F1E09192021E9FF0011124EC56A1
:10403000FD4F4081518162817381848195810E940D
:10404000141D8091920290E00196877099278093C9
:104050009202D9CF0E94821910929302109292027A
:10406000E4ECF2E086E0DF011D928A95E9F72C96F8
:104070000FB6F894DEBF0FBECDBFDF91CF911F9179
:104080000895DF92EF92FF920F931F93CF93DF93E8
:10409000FC01892B09F488C0E12CF12CDD24D39498
:1040A000EF0121968491853709F460C058F4843774
:1040B00008F04EC0843008F068C08130D1F0823002
:1040C00071F172C0883709F45BC050F4863709F487
:1040D00053C0873709F068C08E2D0E942D2352C02F
:1040E0009CE7980F903708F05FC08F770E943A19CD
:1040F0004EC08F010E5F1F4FFE01849190E2980F1A
:10410000983050F48770FD2D01C0FF0F8A95EAF7B3
:104110008F2F0E94332315C00E94CF1814C08F0127
:104120000E5F1F4FFE01849190E2980F983068F463
:104130008770FD2D01C0FF0F8A95EAF78F2F0E942F
:1041400039230E945A23E80122C00E943A19FBCF6A
:10415000CF010296FE01C491CC2361F0EFE9FFE0AC
:104160003197F1F700C00000C150F6CFCF010296A1
:10417000FE01F490EC010BC00E941D23E82E07C045
:104180000E9430230E945A2302C00E94CF188F2D14
:10419000882341F0EFE9FFE03197F1F700C000001C
:1041A0008150F6CFFE017CCFDF91CF911F910F910F
:1041B000FF90EF90DF90089560934A0370934B0354
:1041C00080934C0390934D030C94A823089560931F
:1041D0004E0370934F0380935003909351030C94BC
:1041E000A7230F931F9300914E0310914F0320912B
:1041F000500330915103602B712B822B932B6093D2
:104200004E0370934F0380935003909351031F917B
:104210000F910C94A7230F931F9300914E031091BD
:104220004F03209150033091510360237123822367
:10423000932360934E0370934F03809350039093A6
:1042400051031F910F910C94A7230F931F9300917B
:104250004E0310914F03209150033091510360277A
:1042600071278227932760934E0370934F038093A7
:104270005003909351031F910F910C94A72360E07A
:1042800070E0CB010C94DC200F931F9341E050E0D1
:1042900060E070E08A019B0104C0000F111F221F23
:1042A000331F8A95D2F7C901B8011F910F910C9461
:1042B000DC200F931F9341E050E060E070E004C009
:1042C000440F551F661F771F8A95D2F780914A03C6
:1042D00090914B03A0914C03B0914D038A019B0137
:1042E000082B192B2A2B3B2BC901B8011F910F91C9
:1042F0000C94DC200F931F9341E050E060E070E0ED
:1043000004C0440F551F661F771F8A95D2F740954A
:1043100050956095709580914A0390914B03A091C0
:104320004C03B0914D038A019B01082319232A23D2
:104330003B23C901B8011F910F910C94DC200F930E
:104340001F9341E050E060E070E004C0440F551F4F
:10435000661F771F8A95D2F780914A0390914B038D
:10436000A0914C03B0914D038A019B0108271927A6
:104370002A273B27C901B8011F910F910C94DC201B
:104380000F931F9300914A0310914B0320914C030C
:1043900030914D03602B712B822B932B1F910F912A
:1043A0000C94DC200F931F9300914A0310914B0350
:1043B00020914C0330914D0360237123822393237A
:1043C0001F910F910C94DC200F931F9300914A03CF
:1043D00010914B0320914C0330914D0360277127BE
:1043E000822793271F910F910C94DC2008958F92C0
:1043F0009F92AF92BF92DF92EF92FF920F931F9323
:10440000CF93DF9300D000D01F92CDB7DEB76B8380
:104410007C838D838A018C819D81892B31F01F3FA4
:1044200031F481E04F3F19F403C081E001C080E026
:1044300080FF03C080E090E04DC08B818823D1F1E4
:1044400080904A0390904B03A0904C03B0904D0392
:1044500080914E0390914F03A0915003B09151036E
:10446000882A992AAA2ABB2A8FE1E82EF12CD501A5
:10447000C4010E2C04C0B695A795979587950A940C
:10448000D2F780FD06C081E0E81AF10880F7D12C50
:1044900007C0DE2CB8018E2D0E945F06019799F3AC
:1044A00088E0189FF0011124E653FD4FE00FF11D45
:1044B000D08209C088E0189FF0011124E653FD4F17
:1044C000E00FF11DD08009831A8369817A818D2DD7
:1044D0000E945F060F900F900F900F900F90DF914A
:1044E000CF911F910F91FF90EF90DF90BF90AF9011
:1044F0009F908F90089590911401992379F1909154
:104500001501992359F1982F9695969596959F3177
:10451000A1F0E0911601F0911701E90FF11D8770EC
:1045200021E030E0A90102C0440F551F8A95E2F74F
:10453000CA019181892B818308959091750390FF21
:1045400029C01F928F9388E797E09F938F930E94D3
:1045500056060F900F900F900F900895209116011E
:1045600030911701F90132969FEF40E05191851784
:1045700089F09F3F19F4511101C0942F4F5F4E31C4
:10458000A9F79F3F39F0F901E90FF11D97FDFA9561
:1045900082830895089590911401992381F1909157
:1045A0001501992361F1982F9695969596959F31CF
:1045B000A9F0E0911601F0911701E90FF11D877044
:1045C00021E030E0A90102C0440F551F8A95E2F7AF
:1045D000CA01809591818923818308959091750303
:1045E00090FF1CC01F928F938AE597E09F938F9353
:1045F0000E9456060F900F900F900F900895E09133
:104600001601F09117019F01225E3F4F928189139D
:1046100001C012823196E217F307C1F7089581E0D5
:1046200090E0E0911601F0911701E80FF91F108258
:10463000019680329105A9F7089580917403089539
:1046400090917403892B80937403089580959091C1
:1046500074038923809374030895809374030895E9
:1046600010927403089590917303892B80937303C0
:10467000089580959091730389238093730308951F
:104680001092730308958093520308951092520379
:1046900008958091160190911701FC0131969C01BB
:1046A000205E3F4F80E0919191118F5FE217F307F9
:1046B000D1F70895E0911601F091170180917403EC
:1046C0008083E0911601F09117019081809173032E
:1046D000892B808380915203882361F0E091160139
:1046E000F09117019081892B80830E9449238111C9
:1046F0001092520380911601909117010C940617A5
:10470000909335018093340108958295982F937387
:1047100044E0949F900111248C7C86958695282BEB
:10472000822F8575880F2A7A2695822B0895089501
:10473000CF93DF9300D000D01F92CDB7DEB70F909C
:104740000F900F900F900F90DF91CF9108950895E3
:1047500008950C94501880E0089583B7817F8C6091
:1047600083BF83B7816083BF7894889583B78E7F3A
:1047700083BF0895CF930E9487180E94080B0E9460
:104780008818C0E08C2F0E94EB0A811104C0CF5F13
:10479000C031C1F701C081E0CF9108950E94F10AB4
:1047A0000C9482191F920F920FB60F9211248F93BF
:1047B0009F93AF93BF938091760390917703A091DD
:1047C0007803B09179034196A11DB11D80937603C2
:1047D00090937703A0937803B0937903BF91AF913F
:1047E0009F918F910F900FBE0F901F90189582E0B0
:1047F00084BD93E095BD9AEF97BD80936E000895B8
:104800002FB7F8948091760390917703A091780365
:10481000B09179032FBF08952FB7F8946091760374
:104820007091770380917803909179032FBF089559
:104830009C014FB7F8948091760390917703A091F3
:104840007803B09179034FBF821B930B089578943E
:104850001F920F920FB60F9211248F939F93AF93D5
:10486000BF938091760390917703A0917803B091E4
:1048700079030196A11DB11D809376039093770370
:10488000A0937803B0937903BF91AF919F918F91DB
:104890000F900FBE0F901F9018950E948A15F894E4
:1048A00087E797E7909301088093000887E090EBF3
:1048B000DC018093880390938903A0938A03B093CB
:1048C0008B039CE088E10FB6F894A8958093600074
:1048D0000FBE90936000FFCF80E090E008950895B0
:1048E000CF93C82F1F928F938CE997E09F938F935C
:1048F0000E94560681E090E0A0E0B0E0BC01CD014E
:1049000004C0660F771F881F991FCA95D2F70E94AF
:10491000E7200F900F900F900F90CF910C94821979
:10492000CF938732A8F58E3108F02BC1803109F47E
:104930009FC0F8F4873009F464C0A8F4863009F009
:1049400024C180917503817F8E7F8093750381EAF6
:1049500097E00E94BD0584E89AE00E94BD0581E0D1
:1049600080937A034CC08B30F1F18E3009F46CC027
:104970000CC1863109F4B0C020F4813109F4EDC0D6
:1049800004C1893109F491C08B3109F449C0FDC0DB
:10499000883349F150F4893209F4F1C0853309F4C0
:1049A000EEC0873209F0F1C0EAC0833409F4E7C0F1
:1049B00028F48A3308F4E9C08953E4C0883409F044
:1049C000E4C00E94821983E79AE00E94BD052FEFA0
:1049D00083ED90E3215080409040E1F700C000005B
:1049E0000E944D240CC08CEB97E05CC08AE59AE0F5
:1049F0000E94BD0580917503816080937503C1E0BD
:104A0000C9C080917503C82FC17080FFEFCF86E6C3
:104A10009AE00E94BD0580917503817F8E7F3DC025
:104A20009091750391FBCC27C0F981E0C827892FAD
:104A3000C0FB81F980937503CC2319F08DE49AE0D3
:104A400027C08FE39AE02EC09091750392FBCC278C
:104A5000C0F981E0C827892FC0FB82F980937503D4
:104A6000CC2319F080E39AE013C080E29AE01AC0E8
:104A70009091750393FBCC27C0F981E0C827892F5B
:104A8000C0FB83F980937503CC2351F084E19AE055
:104A90000E94BD05809175038160809375037AC083
:104AA00087E09AE00E94BD05AACF88EF99E00E94B6
:104AB000BD0582ED99E00E94BD058AE899E00E945B
:104AC000BD0582E699E00E94BD0586E199E00E945D
:104AD000BD058AEE98E0E6CF8CED98E00E94BD051A
:104AE0000E94FA161F928F9382EC98E09F938F9307
:104AF0000E945606809114011F928F938BEA98E0D2
:104B00009F938F930E94560680917A021F928F93F3
:104B100088E998E09F938F930E9456068091150133
:104B20001F928F9385E898E09F938F930E9456067B
:104B30000E940C249F938F937F936F938EE698E04F
:104B40009F938F930E9456068DB79EB746960FB6D9
:104B5000F8949EBF0FBE8DBF52CF0E948219C091A4
:104B6000150181E0C827C0931501CC2329F084E604
:104B700098E00E94BD050EC089E598E093CF80E0E3
:104B800001C08D510E9470243ACF87E598E00E94C1
:104B9000BD05C0E08C2FCF91089580E008950C945E
:104BA000CD25CF93C82F80917A03882319F08130C7
:104BB00059F042C0E0911601F091170180818232D4
:104BC00061F08434D9F509C0E0911601F091170124
:104BD0008081823211F0843461F48C2F0E94CF25C1
:104BE000811104C08C2F0E94902424C081E090E0A9
:104BF00021C08C2F0E94CD2581111BC0C43189F0AA
:104C000018F4CB3029F010C0C93259F0C83361F420
:104C100081EA97E00E94BD0588E997E00E94BD0502
:104C200008C010927A030CC086E997E00E94BD0587
:104C300007C081E0817006C010927A0380E002C054
:104C400080E0F8CFCF910895EE0FFF1F0024001CE5
:0E4C50000BBE0790F691E02D0994F894FFCF6B
:104C5E000080FFFF0559010000FFB20E1F0FB50EB9
:104C6E00EA0EB60E0101530340362239C6069006EF
:104C7E006E063506C105DA05F305130600001000B1
:044C8E000800040016
:106800008800EA44E944E244040005000600070069
:10681000080009000A000B000C000D000E000F001C
:1068200010001100120013001400150016001700CC
:10683000180019001A001B001C001D001E001F007C
:10684000200021002200230024002500260027002C
:10685000280029002A002B002C002D002E002F00DC
:10686000300031003200330034003500360037008C
:10687000380039003A003B003C003D003E003F003C
:1068800040004100420043004400450046004700EC
:10689000480049004A004B004C004D004E004F009C
:1068A000500051005200530054005500560057004C
:1068B000580059005A005B005C005D005E005F00FC
:1068C0006000610062006300640065A185006700EC
:1068D000680069006A006B006C006D006E006F005C
:1068E0007000710072007300890087008A008B00BD
:1068F000E000E100E200E300E400E500E600E7007C
:106900000100010001000100EA4401000100E2442D
:106910000100010001000100460001004A004B0097
:10692000010001004700480001000100E9440100A6
:106930000100010001000100010001003A003B00DC
:106940003C003D003E003F0040004100420043004B
:10695000010035004C0039000100440045005200A0
:1069600049000100010050004F0029004D004E0079
:1069700051000100010001000100010001000100BF
:1069800001000100010001000100010001000100FF
:1069900001000100010001000100010001004D00A3
:1069A0004A004E004B0001000100010001000100FF
:1069B00001000100010001000100010001000100CF
:1069C00001000100010001000100010001000100BF
:1069D00001000100010001000100010001000100AF
:1069E0000100010001000100490001000100010057
:1069F000010001000100010001000100010001008F
:00000001FF
